S02B0000433A2F576F726B2F736F6674776172652F4F70656E424C542F5461726765742F44656D6F2F41524DEF
S11300001C190020F10000003D1E00003D1E0000F0
S11300103D1E00003D1E00003D1E00003D1E000070
S11300203D1E00003D1E00003D1E00003D1E000060
S11300303D1E00003D1E00003D1E00003D1E000050
S11300403D1E00003D1E00003D1E00003D1E000040
S11300503D1E00003D1E00003D1E00003D1E000030
S11300603D1E00003D1E00003D1E00003D1E000020
S11300703D1E00003D1E00003D1E00003D1E000010
S11300803D1E00003D1E00003D1E00003D1E000000
S11300903D1E00003D1E00003D1E00003D1E0000F0
S11300A03D1E00003D1E00003D1E00003D1E0000E0
S11300B03D1E00003D1E00003D1E00003D1E0000D0
S11300C03D1E00003D1E00003D1E00003D1E0000C0
S11300D03D1E00003D1E00003D1E00003D1E0000B0
S11300E03D1E00003D1E00003D1E00003D1E0000A0
S11300F02949072291438D4628482949294A00F075
S113010039F8294829492A4A00F034F829482A4963
S11301102A4A00F02FF82A482A492B4A00F02AF8E4
S11301202A482B492B4A00F025F82B482B492C4A06
S113013000F020F82B482C49002200F026F82B4828
S11301402B49091A082903DB0022026004300160EC
S11301501C481D49884205D00268043003B4904706
S113016003BCF7E700208646EC4600200021214A24
S11301709047FEE7884207D0521A05D00378013031
S11301800B700131013AF9D17047884202D00270F4
S11301900130FAE7704700001C19002038640000A1
S11301A00000002002000020F8010000F801000017
S11301B0F057000038640000000000200000002018
S11301C0F0570000F0570000F0570000F05700000F
S11301D0F0570000F0570000F0570000F0570000FF
S11301E036640000040000209C1600209C160020A9
S10B01F01C170020111E000081
S11301F8A0F58013591E012940F20181814A9042D9
S113020800F0FD8002F58073984200F0F88003F551
S11302180071884200F0F3807B4A904200F0EF803E
S113022802F58073984200F0EA8003F50071884271
S113023800F0E580754A904200F0E180744B9842E2
S113024800F0DD8003F11021884200F0D880714A63
S1130258904200F0D480704B984200F0D080591C32
S1130268884200F0CC808A1C904200F0C880131D9C
S1130278984200F0C4800833984200F0C0801033DC
S1130288984200F0BC802033984200F0B880403394
S1130298984200F0B4808033984200F0B0805F49FF
S11302A8884200F0AC804A1C904200F0A880531C9D
S11302B8984200F0A480591C884200F0A0804A1C8F
S11302C8904200F09C80531C984200F09880591C7E
S11302D8884200F094804A1C904200F090804028A4
S11302E800F08D80B0F1102F00F089804C4B9842BB
S11302F800F085804B49884200F081804A1C904276
S11303087DD0531C98427AD0591C884277D0464AEB
S1130318904274D0454B984271D0454988426ED07A
S1130328444A90426BD0444B984268D0434988422F
S113033865D0B0F1101F62D0414A90425FD0414B62
S113034898425CD003F58071884258D0A1F5F872C0
S1130358904254D01032904251D03B4B98424ED0E8
S1130368591C88424BD0394A904248D0384B98425D
S113037845D0591C884242D08A1C90423FD0131D54
S113038898423CD03349884239D04A1C904236D0EE
S1130398314B984233D0591C884230D08A1C904241
S11303A82DD02E4B98422AD0591C884227D04A1C5B
S11303B8904224D0531C984221D0591C88421ED004
S11303C8B0F1202F1BD0264A904218D0082816D006
S11303D8244B984213D02449884210D04A1C904296
S11303E80DD0531C98420AD0591C884207D04A1C85
S11303F8904204D0531CC11A484248417047012016
S1130408704700BF0001100000011010005800F0F0
S113041800401010005400F001000020090800F00A
S113042800400010022000F00010101000011020FD
S1130438004800F080000030005000F01000003048
S1130448014000F000010010021C00F02000003000
S113045801001010040400F001000010031800F05B
S11304680100102000101000005C00F013B50446D1
S1130478FFF7BEFE20B91F4840F2313101F07CFF7E
S113048804F07043B3F1704F1AD1E1B2C4F30724F6
S113049804F57E228B0002F5A06143F0844021F428
S11304A8700340EA43140120206000200190019A5F
S11304B80F2A02D8019B581CF8E70021216018E094
S11304C8220FA1B2C4F3044401FA04F40A4850F810
S11304D822301A6844EA0200186000220192019A44
S11304E80F2A02D80198421CF8E7196821EA040483
S11304F81C601CBD5C580000D458000010B50446AC
S1130508FFF776FE20B9144840F2963101F034FF23
S113051804F07043B3F1704F10D1C4F30721E0B273
S113052801F57E24830004F5C06043F0844220F47E
S1130538700342EA43140122226010BD220FA1B2C3
S1130548C4F3044401FA04F4044850F822301A6845
S113055814431C6010BD00BF5C580000C85800005C
S113056801387FF4FDAF70474E4B2DE9F0411A680E
S1130578044612F0E04F05D018684B490140B1F128
S1130588805F02D1002CC0F28A80484F48483B68FB
S1130598066823F4800545F4006546F400623D606E
S11305A80260980701D5A10703D5DB0719D5E7072A
S11305B817D464F003013D4F0D40002A3D6005DA6D
S11305C806F07000302805D0702802E005F03003EA
S11305D8302B02D14FF4805001E04FF40020FFF794
S11305E8BFFF26F00046334B26F0700141F4006744
S11305F804F4FE62234025F4FE6545EA020847EA4E
S113060803002B4E294F04F0080540EAC505C7F836
S1130618008010203560FFF7A3FF04F4405228F44B
S11306284053134304F4005125F400522248402552
S11306380A43224905604BBF32603B603B6032602D
S113064804F0FC5023F0F86322F0FC5223F0030377
S113065821400243600043EA010307D5184922F404
S11306688002214043F480030A4301E022F08042DF
S113067821050BD44FF4004112480068400601D408
S11306880139F9D123F4006322F4006207480849C8
S1130698036010200A60BDE8F041FFF761BFBDE8C0
S11306A8F08100BF00E00F400000FF7060E00F40E1
S11306B870E00F403000008058E00F400300C0078E
S11306C80000404050E00F405F4B70B51A6810338B
S11306D81B68002BB4BF03F0700102F0300120291D
S11306E837D004D869B1102940F0AB800FE06029F5
S11306F854D070294FD0302940F0A38047F23050AD
S113070856E05249C2F3841051F8200050E0504991
S1130718086810F0E04F44D00C684E482040B0F10F
S1130728805F3ED00C684B4820404B4CA04203D11C
S1130738096888B2022836D04548464904682140E9
S1130748464CA14201D0464832E0006881B251B318
S1130758F9E73F49086810F0E04F26D00C683D4897
S11307682040B0F1805F20D00C683A4820403A4CD1
S1130778A04203D1096888B2022818D03448354900
S113078804682140354CA14201D0364810E0006885
S113079881B261B1F9E74FF4004009E04FF48000F9
S11307A806E0314804E0314802E0314800E03148CD
S11307B8002B02DA13F4006F01E012F4006F28D161
S11307C82D4D2968224D2C6814F0E04F43F6E0744F
S11307D804EA01044FEA541405D02E681D4D35402F
S11307E8B5F1805F05D1023401F01F05604302357D
S11307F804E0604301F01F0501356D00B0FBF5F01E
S113080811F4804F18BF4008090448BF800842F417
S11308188002510216D5002B0DDA590005D51A05A8
S113082803D44000C3F3865201E0C3F3C552531CFA
S1130838B0FBF3F070BDC2F3C353591CB0FBF1F025
S113084870BD002070BD00BF60E00F40F05700008D
S113085800E00F400000FF700000011000000310CA
S11308680024F40000093D00C0E1E400001BB700C7
S113087870383900C0C62D0064E00F40B0F1402F35
S11308885CD02F4B984259D0A3F5A621884255D065
S113089801F5A822904251D0A2F5A62398424DD042
S11308A803F5A821884249D0A1F5A622904245D053
S11308B802F5A823984241D0A3F55C3188423DD083
S11308C801F56032904239D0A2F55C33984235D0B4
S11308D803F56031884231D0A1F55C3290422DD0C5
S11308E802F56033984229D0A3F55C31884225D0BB
S11308F801F56032904221D0A2F5083398421DD008
S113090803F50C31884219D001F58052904215D074
S113091802F58053984211D003F5805188420DD0D6
S113092801F58052904209D002F58053984205D0CF
S113093803F58051421A50425041704701207047D4
S11309480080054070B504460D461646FFF796FF2D
S113095820B911484FF4907101F00EFD022E04D90C
S11309680D484FF4917101F007FDD4F8003416F0E6
S1130978010F14BF2B43AB4304F580621360D4F812
S1130988200416F0020F04F5846114BF054320EA1D
S113099805050D6070BD00BFE0580000F8B50446B9
S11309A80D4617461E46FFF769FF20B93C4840F23A
S11309B8FF1101F0E1FC7B1E012B08D9042F06D09E
S11309C80C2F04D0364840F2032101F0D5FC082E40
S11309D80BD00A2E09D00C2E07D0092E05D026B12B
S11309E82F484FF4027101F0C7FCD4F8000517F042
S11309F8010F14BF2843A84304F5A0621060D4F87B
S1130A08041517F0020F14BF2943A94304F2045331
S1130A181960D4F8080517F0040F14BF2843A84335
S1130A2804F5A1621060D4F8181517F0080F14BF64
S1130A382943A94304F5A3631960D4F80C0516F0F7
S1130A48010F14BF2843A84304F20C521060D4F8D1
S1130A58101516F0020F14BF2943A94304F5A26325
S1130A681960D4F8140516F0040F14BF2843A843DA
S1130A7804F214521060D4F81C1516F0080F04F28E
S1130A881C5314BF2943A943196004F5A560D4F87D
S1130A9828250EB9154301E022EA05050560F8BDCD
S1130AA8E058000070B504460D461646FFF7E6FE0A
S1130AB820B9044840F2853101F05EFC44F8256011
S1130AC870BD00BFE058000070B505460C46FFF73E
S1130AD8D5FE20B9084840F2524101F04DFC2846A1
S1130AE821460222FFF72EFF284621460422082326
S1130AF8BDE87040FFF752BFE058000038B505461E
S1130B080C46FFF7BBFE20B9084840F2F14101F05A
S1130B1833FC2846214601220823FFF73FFF2846D5
S1130B2821460122BDE83840FFF70CBFE058000019
S1130B3870B505460C46FFF7A1FE20B9084840F2F7
S1130B48966101F019FC284621460222FFF7FAFEB5
S1130B582846214601220823BDE87040FFF71EBF3E
S1130B68E058000070B505460C46FFF787FE20B92B
S1130B78084840F2EA6101F0FFFB284621460222B8
S1130B88FFF7E0FE2846214601220823BDE870400D
S1130B98FFF704BFE0580000830510B5044603D0EE
S1130BA80D489C2101F0E8FB0C4B40F601221A6029
S1130BB80B4843F8144C143B0833186019688A0727
S1130BC8FCD4084A40F6012013681840002814BFD2
S1130BD84FF0FF30002010BD4959000014D00F40D9
S1130BE8020042A40CD00F4070B50C46A10706467B
S1130BF8154603D02748DF2101F0BEFBAA0703D01E
S1130C082448E02101F0B8FB234B42F20162234857
S1130C181A600168CB0719D423462DE075B1204A20
S1130C28043D881853F8041B0160A11B5A1812F0DC
S1130C387C01F3D11B4800680028EFD01A4C1B4EE6
S1130C4826602168C807FCD414461E462DB1184BEB
S1130C5824F07F0018603346E7E7164842F2016241
S1130C6801680A40002A14BF4FF0FF30002070BD0D
S1130C780268D107FCD404332A199A42EDD00C48EF
S1130C88311B0360C8580C4A08491060101D0160E4
S1130C98EEE700BF4959000014D00F40A0E10F400F
S1130CA800D10F4030D00F4020D00F40010042A4A3
S1130CB800D00F400CD00F4004D00F4038B50C467C
S1130CC8054620B910484FF4217101F055FB24B9A9
S1130CD80D4840F2852101F04FFB0C4B1A6812F0C5
S1130CE8E04F0DD018680A490140B1F1805F07D080
S1130CF8084B09481A682A6001680020216038BD39
S1130D084FF0FF3038BD00BF4959000000E00F40E4
S1130D180000FF70E0E10F40E4E10F40114B9842FE
S1130D281DD003F58051884219D001F580529042B4
S1130D3815D002F58053984211D003F580518842AA
S1130D480DD001F58052904209D002F580539842A3
S1130D5805D003F58051421A504250417047012092
S1130D68704700BF00C0004010B50446FFF7D6FF27
S1130D7820B908484FF4FB7101F0FEFAE36A43F026
S1130D881000E062216B41F4407242F001032363D6
S1130D9810BD00BFB659000010B50446FFF7BEFFEA
S1130DA820B9094840F2162101F0E6FAA3691907A7
S1130DB8FCD4E06A20F01001E162226B22F4407353
S1130DC823F00100206310BDB6590000F8B50446AD
S1130DD80E4615461F46FFF7A1FF20B92A484FF4CF
S1130DE8B07101F0C9FA25B9274840F2611101F040
S1130DF8C3FA264A136813F0E04F1CD0116824483C
S1130E080840B0F1805F16D0136821492148194081
S1130E18814203D1126893B2022B0CD01B481C4A9E
S1130E2801681D4B0A409A4201D0082204E0006878
S1130E3881B20029F9D110226A43964204D2124899
S1130E484FF4B17101F098FA2046FFF7A5FFB6EB0D
S1130E58051F236B04D243F0200121636D0802E0CF
S1130E6823F020002063F600B6FBF5F56A1C002089
S1130E78D309C2F345056362A562E762A06120460F
S1130E88BDE8F840FFF770BFB659000000E00F4016
S1130E980000FF70000001100000031010B50446A4
S1130EA8FFF73CFF20B9054840F2554101F064FAC8
S1130EB8A06980F02001C1F3401010BDB6590000AC
S1130EC810B50446FFF72AFF20B9064840F27641D8
S1130ED801F052FAA369D80654BF20684FF0FF30D6
S1130EE810BD00BFB659000038B504460D46FFF7DB
S1130EF815FF20B9064840F2C94101F03DFAA3693B
S1130F089A0602D42560012038BD002038BD00BFF0
S1130F18B659000010B50446FFF700FF20B904488D
S1130F2840F23B5101F028FAA069C0F3C00010BD9B
S1130F38B6590000094B98420DD003F580518842F8
S1130F4809D001F58052904205D002F58053C11AA8
S1130F584842484170470120704700BF0080004064
S1130F682DE9F843089F0646884614461D46DDF8D1
S1130F782490FFF7DFFF18B92C48CC2101F0FCF9C5
S1130F886CB1022C0BD0012C09D0032C07D0102CE7
S1130F9805D0202C03D02548D22101F0EDF9022DEB
S1130FA804D92248D52101F0E7F908E03DB9B7EBA7
S1130FB8580F09D91D48D72101F0DEF904E00C23A4
S1130FC8B8FBF3F08742F5D8B8FBF7F7B7F57E4FCF
S1130FD803D91648D82101F0CFF9A9F104010C2945
S1130FE803D91248D92101F0C7F9022D02D025B13D
S1130FF8002500E00825042200E02A461543756010
S113100800230233B7FBF3F0411EFF29F9D8A201EC
S1131018336104F03004D3B21C4309F1FF3C44EAC1
S11310280C0949EA01203060BDE8F883225A00001F
S113103810B50446FFF77EFF20B905484FF48571C3
S113104801F09AF9636843F00200606010BD00BFC4
S1131058225A000010B50446FFF76CFF20B9054872
S113106840F2231101F088F9636823F002006060FC
S113107810BD00BF225A000038B504460D46FFF7DC
S113108859FF20B90B4840F2232101F075F9236870
S11310986FF0010203F00F0002FA00F1294204D0B4
S11310A8044840F2252101F067F9E3689A07FCD562
S11310B8A56038BD225A000038B504460D46FFF72E
S11310C839FF20B9054840F27F2101F055F9E3685A
S11310D85907FCD5A068286038BD00BF225A000013
S11310E80369F0B500F1100C9EB20546180C1C0EED
S11310F80870B01F4C7002239042B4BF04461446D3
S1131108E71E9F4204DDDCF80070CF500433F7E794
S1131118A34218DABB422D6907D1CD54CB18290A4A
S11311282D0C59709D70631C0DE0A71EBB4205D1A0
S1131138CD54C9182D0A4D70A31C04E0671EBB4288
S113114801D1CD54E31CB11E8B4203DADCF8001044
S11311580433F8E79042C8BF4042F0BD30B54B783D
S11311680C781D0645EA0443A2F10E0423430361E7
S113117800F110050223D41E9C4203DDCC5804332D
S11311882C60F8E7934218D0A34208D1CC5CCB1862
S113119899785B781B0243EA014121430CE0941ED1
S11311A8A34205D1CC5CCB18597844EA012103E069
S11311B8541EA34201D1C95C016101218163104617
S11311C830BD000038B5074B044698420D4603D09D
S11311D805485D2101F0D0F80448B5FBF0F1CDB223
S11311E8656238BD008004408A5A0000404B4C00B8
S11311F838B5134B044698420D4603D01148A6212E
S113120801F0BAF825F4873020F0160119B10D4819
S1131218AA2101F0B1F8E268E8B222F01603034308
S1131228E360A168C5F3072221F00E031343A3600A
S1131238E06BC5F3074520F001010D43E56338BDB4
S1131248008004408A5A0000144B37B5984205467A
S11312580C4604D0124840F2131101F08DF824B959
S11312680F484FF48A7101F087F820786178A278E2
S1131278E3788DF805108DF804008DF806208DF8B4
S113128807300198002168612279637901918DF80A
S113129804208DF805300198A8613EBD0080044003
S11312A88A5A00000D4B10B59842044604D00C48E5
S11312B840F2691101F060F8A06840F01001A160E3
S11312C8A26842F00103A360E06840F00101E16014
S11312D8A26842F01003A36010BD00BF0080044060
S11312E88A5A0000124B70B5984204460E461546B9
S11312F804D0104840F28F2101F03EF826B90D4879
S11313084FF4247101F038F8002D04DC094840F248
S1131318912101F031F8606B10F03F0006D02046AF
S113132831462A46BDE87040FFF7DABE70BD00BFFB
S1131338008004408A5A0000144B70B59842054650
S11313480E46144604D0124840F29E3101F014F8B7
S113135826B90F4840F29F3101F00EF8002C04DC46
S11313680B484FF4687101F007F8A86BC107FCD467
S113137840F2FE718C4201DD604270BD2846314660
S11313882246BDE87040FFF7E9BE00BF0080044074
S11313988A5A000038B50B4B044698420D4604D0CF
S11313A8094840F2474100F0E7FF35F07F0304D0D5
S11313B8054840F24A4100F0DFFF606820EA05056D
S11313C8656038BD008004408A5A000038B5074B70
S11313D8044698420D4604D0054840F26A4100F09C
S11313E8CBFF20680DB16168084038BD0080044017
S11313F88A5A000038B50A4B044698420D4604D070
S1131408084840F29F4100F0B7FF35F07F0304D04D
S1131418044840F2A24100F0AFFF256038BD00BF88
S1131428008004408A5A000038B50D4B044698429F
S11314380D4604D00B4840F2125100F09DFF226A79
S113144804F12001D207FAD4E800C5B245F0010539
S11314580D600B68D807FCD4216B88B238BD00BF77
S1131468008004408A5A000013B5064C0146204601
S1131478FFF702FE204601A9FFF71EFE9DF80400AF
S11314881CBD00BF0080004038B500F0DBFE00F54D
S1131498FA75FF20FFF7E8FFFF28044603D000F0A1
S11314A8D1FEA842F5D3B4F1FF035842584138BDE0
S11314B8012108B504480A46FFF7F4FAFF20BDE8FD
S11314C80840FFF7D1BF00BF0070004010B50121EC
S11314D800220848FFF7E6FAFF20FFF7C5FFFFF7E9
S11314E8D3FF044618B9FFF7E3FF204610BD0120D7
S11314F810BD00BF0070004038B50D460106044613
S113150807D537200021FFF7F7FF012832D804F068
S11315187F04FFF7CDFFFFF7D9FF50B344F0400035
S1131528FFF7A2FF280EFFF79FFFC5F30740FFF759
S11315389BFFC5F30720FFF797FFE8B2FFF794FF77
S113154824B1082C0CBF8720012000E09520FFF768
S11315588BFF0C2C02D1FF20FFF786FF0A24FF2003
S1131568FFF782FF020605D5013C14F0FF04F6D10B
S113157838BDFF2038BD38B505460024285DFFF77F
S113158873FF2B1958780234FFF76EFFB4F5007F08
S1131598F4D1FF20FFF768FFFF20FFF765FFFF2066
S11315A8FFF762FF00F01F00B0F1050EDEF1000145
S11315B851EB0E0038BD70B505460E4600F042FEEC
S11315C800F16404FF20FFF74FFFFF2805D100F066
S11315D839FEA042F6D3002070BDFE28FBD1AC1C16
S11315E8FF20FFF741FF04F8020CFF20FFF73CFF40
S11315F8AB1904F8010C0234981CA042F0D1FF2066
S1131608FFF732FFFF20FFF72FFF012070BD000016
S11316187FB5002840F0FA807E490C7804F0020077
S1131628C4B2002C40F0F0807B48FEF767FF7B488B
S1131638FEF764FF7A48FEF761FF4FF0402034213B
S1131648FFF776FA77480121FFF758FA4FF0402060
S1131658342102220A23FFF7A1F90A237148012140
S11316680222FFF79BF901210A466E48FFF71AFA8E
S1131678FFF72AF86C4B4FF0080C8DE80810014668
S1131688234622466948FFF76BFC6848FFF7D0FCFD
S113169801210A466348FFF705FA4FF0402020214C
S11316A8FFF72CFA20214FF040200A46FFF7FAF9F9
S11316B80A24FF215D48FFF7DFFC5C4803A9FFF714
S11316C8FBFC013CF5D120214FF04020FFF730FA14
S11316D8012154482246FFF7E5F920462146FFF741
S11316E80BFF0128064601D0002466E000F0AAFD9D
S11316F84FF4D57100F57A750820FFF7FDFE01282F
S113170839D1FF20FFF7B0FE02AB18550134042C81
S1131718F7D19DF80A100129E6D19DF80B20AA2AD1
S1131728E2D100F08FFDA84204D300F08BFDA8425B
S1131738DAD207E0A9204FF08041FFF7DDFE002848
S1131748EFD1F2E73A200021FFF7D6FE0028CBD1EB
S11317580446FF20FFF788FE02AB18550134042C19
S1131768F7D19DF8080000F04001CAB2002A0CBF66
S113177804240C2421E0A9202146FFF7BDFE0128FA
S113178802D80224A92600E0344600F05BFDA842F2
S11317980CD300F057FDA842A6D210204FF40071D4
S11317A8FFF7AAFE002818BF002406E030460021EF
S11317B8FFF7A2FE0028E8D1EBE71D4B1C60FFF7FA
S11317C877FE14480178DCB101F0FE040470174870
S11317D8FFF740FCFEF778FF4408FEF775FF154B4A
S11317E80146002208209C4294BF00940093019073
S11317F813460E48FFF7B4FB0C48FFF719FC02E048
S113180841F0010202700349087800E0012004B0A5
S113181870BD00BF0000002010000010010000206F
S11318280800002000700040801A06000080004074
S11318380400002020BCBE0010B9024B1878704781
S1131848012070470000002038B50D461C4611469B
S1131858002834D1002B32D01B4B1878C20730D45F
S11318681A4A13681B0758BF4902012C0DD11120CD
S1131878FFF742FEE8B928464FF40071FFF79BFED4
S1131888D0F1010438BF002413E01220FFF734FE1E
S113189878B928464FF40071FFF78DFE28B1013C52
S11318A814F0FF0405F50075F3D10C200021FFF7AF
S11318B823FEFFF7FDFD201C18BF012038BD0420BE
S11318C838BD032038BD00BF0000002004000020FC
S11318D870B50D4616461C46002851D1002B4FD032
S11318E82A4B1A78D0074DD4187800F00401CBB2EB
S11318F8002B49D1264A1068010758BF7602012CEB
S113190815D118203146FFF7F7FD08B1012431E05D
S1131918FFF7BAFD0028F9D0FE20FFF7A5FD2846F9
S1131928FFF729FED0F1010438BF002422E010F0AB
S1131938060F03D097202146FFF7DEFD1920314614
S1131948FFF7DAFDB0B9FFF79FFD60B1FC20FFF7A0
S11319588BFD2846FFF70FFE28B1013C14F0FF0465
S113196805F50075EFD1FFF78FFD0028CED0FD20D7
S1131978FFF77AFDFFF79CFD201C18BF012070BDFE
S1131988042070BD032070BD022070BD000000203B
S113199804000020F0B5154685B0002840F0EE801C
S11319A8794B1878C30700F1EB800E2900F2E28026
S11319B8DFE811F00F001200E0005200E000E00040
S11319C8E000E000E000E000A700AB00AD00B700D5
S11319D8C800FFF77BFDC8E009200021FFF78CFD54
S11319E8044608B10124C6E068461021FFF7E3FD68
S11319F80028F7D09DF800109DF807308A09012ABD
S1131A080CD103F03F009DF808109DF8093002043A
S1131A18501C03EB0122801880023FE09DF8080067
S1131A289DF80620990001EB901302F0030003EBE4
S1131A3880219DF805309DF80A20481C03F00F0109
S1131A4801EBD2139DF8091001F0030203EB4203E2
S1131A58D91F00FA01F021E04C4E316811F004015D
S1131A681ED08D200021FFF747FD0028BAD1FF20A2
S1131A78FFF7FAFC68461021FFF79DFD0028B1D056
S1131A883024FF20FFF7F0FC611E11F0FF04F8D1A9
S1131A989DF80A201023100903FA00F028606AE070
S1131AA80920FFF729FD074600289BD16846102125
S1131AB8FFF781FD002895D032689DF80A0012F0DE
S1131AC8020410D000F03F049DF80B00C30903EB97
S1131AD844019DF80D404A1CA009431E02FA03F272
S1131AE83C462A6047E09DF80B30C0F3840103F0BC
S1131AF803025B09481C03EBC2014A1C42432A60E7
S1131B0839E0224B186810701AE0092000E00A2016
S1131B180021FFF7F1FC00287FF464AF2846102168
S1131B2821E03A200021FFF7E7FC00287FF45AAFB0
S1131B380446FF20FFF798FC28550134042CF8D1FB
S1131B48002418E011490A6854077FF54BAF8D202B
S1131B580021FFF7D1FC00287FF444AFFF20FFF7F2
S1131B6883FC28464021FFF726FDD0F1010438BF45
S1131B78002400E00424FFF79BFC02E0042400E0B6
S1131B880324204605B0F0BD000000200400002016
S1131B98004870470000AA4210B5044C2046FEF7DE
S1131BA8ADFC2046BDE81040FEF760BC0050102094
S1131BB830B53E4885B0FEF7A1FC3D480C21FEF740
S1131BC883FF3C487F21FFF7E5FB00213948FFF7F5
S1131BD8FDFB01463748FFF70DFCFEF775FD01468E
S1131BE83448FFF7EFFA16213248FFF701FB314872
S1131BF8FFF758FB01212F48FFF716FC044600F0B5
S1131C0821FB00F59C5000F10805600708D4012168
S1131C182848FFF709FC044600F014FBA842F4D353
S1131C280021082369208DF80910452127228DF801
S1131C3808308DF80B005B238DF80D10684601A958
S1131C488DF80A208DF80C30FFF738F8009A531CE9
S1131C5812D00198411C0FD0130A110C8DF80820DA
S1131C688DF80B00020A000C8DF809308DF80A1063
S1131C788DF80C208DF80D000E4802A9FFF7E4FA40
S1131C880D4B9DF808109DF809209DF80A0019705D
S1131C985A7098709DF80B109DF80C209DF80D0053
S1131CA8D9701A71587105B030BD00BF20000020EA
S1131CB800500240008004401A16002010B500218C
S1131CC80948FFF783FB044621460748FFF792FBC0
S1131CD814F0010007D00448044940F24262BDE808
S1131CE81040FFF7FFBA10BD00800440C20F002067
S1131CF8024B034803491A88FFF71EBBB80F00209C
S1131D0800800440C20F002000B589B00021684655
S1131D18202203F05FFD0848694602F023FC40B91D
S1131D28009838B19DF8080080F01001C1F3001044
S1131D3800E0002009B000BDF75A000000487047D1
S1131D48F75A000010B5074C0023204606490A221A
S1131D5884F8243202F0E0F810B9012084F824024F
S1131D6810BD00BF08000020125B000010B50C482D
S1131D7890F82432012B01D102F04FFB00F062FAF3
S1131D8800F164040748FFF7C5F8012803D100F0FF
S1131D9859FAA042F6D90448BDE8104002F006BC3E
S1131DA80800002000C00040F75A0000034890F8DB
S1131DB82432012B01D102F030BB70470800002007
S1131DC838B50F4C054694F82432012B0AD1214624
S1131DD802F088FC002805DA002084F82402204652
S1131DE802F01BFB6C1E14F8011F41B10548FFF7F4
S1131DF87BF80448FFF752F80028FAD0F3E738BD17
S1131E080800002000C0004008B50848FEF7ACFBF5
S1131E180748FEF773FB4FF040200321FEF7A2FEAC
S1131E2800F0E2FA00F0F1FAFCE700BF8003C00119
S1131E38010000200148382100F09EBA1F5B000011
S1131E4872B6704762B67047FFF7FABF10B500F074
S1131E58C8F988B100F014FB00F0E0F900F0C3F908
S1131E68064B20F0604020F07F01196000F0BBF9B8
S1131E784468FFF7E7FFA04710BD00BF08ED00E086
S1131E88F8B505460E4617460024A3B29F4205D06E
S1131E98A05D605500F025FB0134F6E7F8BD0000AD
S1131EA870B500240646254600F01BFB094BE25892
S1131EB8964209D3191948681218964204D20C217B
S1131EC801FB0535287A70BD0C340135C02CEBD1E3
S1131ED8FF2070BDA45B00002DE9F34105460068AE
S1131EE8FFF7DEFFFF2801D100201AE000242B1998
S1131EF858682F6802AE46F8040D04EB070800F092
S1131F08F0FA304641460422FEF76EFE0028EBD173
S1131F18E25901998A42E7D10434B4F5007FE6D145
S1131F280120BDE8FC81000038B5104B04469842F6
S1131F380D4606D0B1F5004F05D0FFF7CDFF18B90F
S1131F4810E00B4C00E01C46EB050BD12068A842BE
S1131F5809D0204640F8045B29464FF40072FFF785
S1131F688FFF00E00024204638BD00BF3002002067
S1131F78340400202DE9F8439946036821F4FF75D9
S1131F88013304460E46904625F0010506D140F873
S1131F98045B29464FF40072FFF772FF2068A842D9
S1131FA808D020462946FFF7BFFF044610B9002091
S1131FB8BDE8F88321684746761AA219161D00F071
S1131FC890FA231DF01AB0F5007F08D3204605F5D2
S1131FD80071FFF7A9FF04460028E8D0061D17F88A
S1131FE8011B08EB0902974206F8011BE7D10120FF
S1131FF8BDE8F883034A04484FF0FF3313600360D5
S1132008704700BF340400203002002070B5044635
S11320180D461646FFF744FFFF2815D0601E4019E9
S1132028FFF73EFFFF280FD024F4FF7323F00101CC
S1132038B1F5004F0CBF05480548214632462B46EA
S1132048BDE87040FFF796BF002070BD3002002045
S113205834040020F8B505460E46FFF721FF044670
S1132068681E8019FFF71CFFFF2C05464DD0FF287A
S11320784BD0844249D8032C47D9132845D8002685
S113208800F02FFA224B0C2202FB06310F7AA742EA
S113209801D10C6804E00136102EF1D14FF0FF3461
S11320A8002700F01EFA1A4A0C2000FB0723197AAD
S11320B8A94201D11F6804E00137102FF1D14FF074
S11320C8FF37002600F00DFA114A0C2000FB062306
S11320D8197AA94201D15D6803E00136102EF1D1C5
S11320E800253F1B7819C0F38F270025BD420AD26B
S11320F800F0F7F92046FEF74FFD04F5806420B997
S11321086A1C95B2F2E70120F8BD0020F8BD00BFB3
S1132118A45B00000E4B07B51A68013216D0586844
S11321289968DA680918881819695A694018811869
S11321389869DB690A18D118484202AA42F8040DC2
S1132148042148F2F000FFF761FF00E001200EBD12
S11321583002002048F204034FF400410A6818686A
S113216848F2080319688018421848F20C000368FA
S1132178D11848F21002106848F214031A680918B2
S1132188881848F218010B68C21848F2F000016870
S11321985318D3F1010038BF002070470A4808B526
S11321A80368013305D1094801684B1C06D1012095
S11321B808BDFFF791FE0028F5D108BDFFF78CFE96
S11321C8003018BF012008BD30020020340400206C
S11321D84FF400407047FFF70DBFFFF717BFFFF735
S11321E839BFFFF7B7BFFFF7F3BF08B5FFF792FF93
S11321F818B1BDE80840FFF7D1BF08BD054B002260
S11322084CF24F3105201A6059609A601860024BED
S11322181A60704710E000E038060020014B0022E5
S11322281A60704710E000E0044B1868C30303D534
S113223803490A68531C0B60704700BF10E000E0B4
S11322483806002008B5FFF7EFFF014B186808BDF2
S11322583806002010B50748FEF750F9FEF734FA9F
S1132268014605484FF461426023BDE81040FEF77B
S1132278ADBD00BF0100001000C00040402970B58A
S113228806460D4603D916485B2100F075F8154833
S11322982946FEF729FE30B11248FEF7FFFD30B992
S11322A800F01FF9F8E70E485F2100F065F80024F4
S11322B8A3B2AB4213D200F014F90A48315DFEF719
S11322C813FE30B10748FEF7E9FD30B900F009F90B
S11322D8F8E70348682100F04FF80134E8E770BDD7
S11322E8645C000000C00040F8B51E4C0646257822
S11322F8A5B91D48FEF7E4FD421C01D10020F8BD34
S11323081A4AC0B210700028F8D0FFF79BFF184B88
S11323181849186001200D702070EFE7154D124818
S11323282F78FEF7CDFD0137431C10D00F49C8554F
S11323382878421CD3B20A782B709A42DED13046F0
S11323480131FFF79DFD002121700120F8BDFFF741
S113235879FF074B196864318842CFD9002020706F
S1132368F8BD00BF7E06002000C000403C060020E7
S1132378800600207D06002008B500F0B2F8FCE7CE
S113238810B500F0ABF8012818D000F053FAA8B142
S11323980B4C2378012B11D1FFF754FF09490A6824
S11323A802F51C531033834208D80020207000F033
S11323B84BFA18B9BDE81040FFF748BD10BD00BF7F
S11323C8840600208806002008B5054B01221A70EF
S11323D8FFF738FF03490860BDE80840FFF7D0BF9E
S11323E8840600208806002008B5FFF72DFD00F0BC
S11323F877F8FFF703FFFFF7EEFE00F005FA00F0A9
S113240811F8BDE80840FFF7DFBF08B500F069F828
S1132418FFF70AFF00F002FB00F014F8BDE80840DB
S1132428FFF7AEBF10B5064C00F066F8FFF712FFD1
S11324380023237003F0D2F80320207010BD00BFDE
S11324480100002008B50C48FFF74EFF012805D10C
S11324580A4B002208481A7000F06CF8064803F08A
S11324680FF9012807D10549032008700248BDE87F
S1132478084000F05FB808BD8C0600200100002069
S1132488704700000A4B70B51A7806460C461D467C
S113249812B9C9B2FFF7F2FE2878032803D13046EF
S11324A8E1B203F0D1F8BDE8704000F03BB800BFDA
S11324B801000020034B1878411E01298CBF4020DD
S11324C80020704701000020034B1878411E0129A1
S11324D88CBF4020002070470100002000F01AB88B
S11324E870477047034BFE2218710220DA70A3F874
S11324F844007047CC060020054B00221A709A64E9
S113250883F84320A3F844209A705A70704700BF98
S1132518CC060020024B1878003018BF0120704701
S1132528CC060020024B002283F84320704700BFEA
S1132538CC060020F8B506780546FF2E824C19D142
S113254800F078F908B91020E4E0002301251020F0
S1132558637063712570E6702071FFF7ABFFA0719B
S1132568FFF7B2FFE071FFF7AFFF010A217265724E
S1132578A57281E02778012F40F0E480F32E57D02C
S11325881FD8CF2E00F0BC8006D8C92E00F0858055
S1132598CC2E40F0BE80BAE0D12E00F0AB80C0F063
S11325A88E80D22E40F0B5800025FF21E170257180
S11325B86571FFF77FFFE571A071257265720722C7
S11325C829E0FA2E4DD00AD8F52E11D026D3F62EAE
S11325D840F09F80FF21E1704268A26494E0FD2EE0
S11325E84CD0FE2E55D0FC2E40F09380002091E074
S11325F8FFF760FF6A78904201DC22208AE0A16C30
S1132608201DFFF73DFCFF20E070A26C69788B1851
S1132618A3646878421CA4F844207DE0FFF74AFFCD
S11326286B789842E9DD6968201DA1646A78E8E757
S1132638FF22E270A36C446800221C19A34204D050
S113264813F8010B1118CAB2F8E73F4B0021C3F87D
S1132658072001200822187159719971A3F84420A0
S11326685AE03A4B0020FF220721E270A36420714C
S11326786071A071C4F807100822CCE761780020C3
S1132688FF23E37020716171A071E071207206224A
S1132698C1E700212170617034E0A66CFFF70AFFDE
S11326A86A1C411E3046FFF798FD80B3FF23A56CD2
S11326B8E370FFF7FFFE013D2818A06424E0FFF74C
S11326C8F9FE6B780138984297DDFF21E170A4F890
S11326D84470697819B9FFF788FDE8B917E01A4C0E
S11326E8AA1CA06CFFF779FD88B16A78A06C13184E
S11326F8A36411E0A06C6968FFF771FD10B906E0E6
S1132708FFF7A4FBFF22E270A4F8447004E0312030
S113271800E02020FFF7E6FE0B4C94F84320012A42
S113272802D11020FFF7DEFEB4F8441006480BB2BD
S1132738002B07DD012280F843200330BDE8F84070
S1132748FFF7A0BEF8BD00BFCC060020DB5C00008C
S113275870B5002506462C46705D03F025F8C0B216
S1132768A0F13003DAB2162A10D8A0F13A010629EA
S11327780CD9092A84BFA0F13702D2B2013502EB81
S11327880414022D04F0FF0401D0E5E700242046D8
S113279870BD000010B503460B4819460A24B1FB66
S11327A8F4F1024601300029F8D102F801190A248B
S11327B8B3FBF4F104FB11333033104602F801394A
S11327C80B460029F3D110BD1907002038B50309B9
S11327D8092B05460C46184601D9373003E030303A
S11327E802F0E2FFC0B2207005F00F00092801D9F9
S11327F8373003E0303002F0D7FFC0B260700020F9
S1132808A070204638BD000008B5074B00200749D2
S1132818187001F071FB28B105487721BDE808401C
S1132828FFF7AABD08BD00BF5807002064070020B1
S1132838E35C0000034B1878D0F1010038BF002096
S1132848704700BF5807002010B5FFF747FE01285E
S113285801D1002010BD054C2378002BF9D1FFF7D6
S113286853FA0128F5D1207010BD00BF5807002085
S113287810B50446007802F097FF532801D00320CE
S113288810BD607802F08AFF0028F8D060783128FB
S113289806D0322806D0332814BF0320022010BDE6
S11328A8002010BD012010BDF8B505460230FFF721
S11328B84FFF04350446074600262846FFF748FF1D
S11328C8013EB6B2BB1999B2201802350129C4B227
S11328D8F3D82846FFF73CFFE243D4B2231A584200
S11328E85841F8BD2DE9F041044616460D4601B19C
S11328F820B9494840F23121FFF73EFD2046FFF751
S1132908B7FF0328074600F082802046FFF7CCFF74
S1132918002879D0012F23D002D3022F77D146E0A3
S1132928A01CFFF715FF8046201DFFF711FF0702C3
S11329382F60A01DFFF70CFF38182860A8F10305C5
S11329480834ADB2002E63D0002729B28F425FDA73
S11329582046FFF7FDFEF05501370234BFB2F4E715
S1132968A01CFFF7F5FE8046201DFFF7F1FE0704C3
S11329782F60A01DFFF7ECFE07EB00272F6004F182
S11329880800FFF7E5FEA8F104023B182B600A349F
S113299895B2002E3CD0002728B2874238DA204668
S11329A8FFF7D6FE791CF05502348FB2F4E7A01C69
S11329B8FFF7CEFE8046201DFFF7CAFE07062F60EC
S11329C8A01DFFF7C5FE07EB00472F6004F10800C0
S11329D8FFF7BEFE07EB00272F6004F10A00FFF79C
S11329E8B7FEA8F10501381828600C348DB27EB101
S11329F800272BB29F420BDA2046FFF7A9FE7A1C68
S1132A08F055023497B2F4E74FF6FF7500E000255D
S1132A1828B2BDE8F08100BFE35C00002DE9F04175
S1132A28A54E3578002D00F08B81012D26D1FFF7B6
S1132A3889F9A248FFF7C4F9A148FFF7C1F9FFF7DC
S1132A487DF92A4601469F4801F066FA044638B1E2
S1132A589D48FFF7B5F92846BDE8F041FFF7A6B948
S1132A689A48FFF7ADF99A48FFF7AAF99948FFF78A
S1132A78A7F99948022304604460BCE0022D40F0A1
S1132A888D80964F964C4FF48071204607F50D7251
S1132A9801F0ECFD97F93A12002901DA8A48A0E01E
S1132AA8F0B10022204604F5C071FFF71BFF421C59
S1132AB804D18548FFF784F9032095E000280FDD49
S1132AC8854D696821B9D4F880116860296007E0E8
S1132AD8D4F880312C684018A34238BF2B60686052
S1132AE87E4DD5F83C22D5F840329A4240F02881F0
S1132AF805F50D70002101F097FC70B17248FFF7DD
S1132B085FF90420FFF752F905F50D7001F085FC13
S1132B18694A00211170BDE8F0816F4C6B48FFF7DA
S1132B284FF97048FFF74CF96068FFF733FE6E48B9
S1132B38FFF746F96D48FFF743F9E0786A49FFF76C
S1132B4845FEA0786A49FFF741FE60786949FFF7B6
S1132B583DFE69492078FFF739FE6348FFF730F9ED
S1132B686648FFF72DF994E80300FFF738FB524C49
S1132B78064660B95448FFF723F90520FFF716F90C
S1132B8805F50D7001F049FC2670BDE8F0814F4849
S1132B98FFF716F903202070BDE8F081032D40F0FB
S1132BA8CF804E4F4E4C4FF48071204607F50D727E
S1132BB801F05CFD97F93A32002B04DA5048FFF72C
S1132BC8FFF8022010E0002859D0204604F5C0710F
S1132BD804F58072FFF786FEB0F1FF3F80460DD101
S1132BE84848FFF7EDF82846FFF7E0F807F50D70B9
S1132BF801F013FC00233370BDE8F08100283EDDAA
S1132C084148FFF7DDF84046FFF7C4FD3648FFF7B3
S1132C18D7F83E48FFF7D4F894F883013249FFF710
S1132C28D5FD94F882013249FFF7D0FD94F881016B
S1132C383049FFF7CBFD304994F88001FFF7C6FD12
S1132C482948FFF7BDF82D48FFF7BAF8D4F88001F2
S1132C5804F580724146FFF7C0FA044660B91A4881
S1132C68FFF7AEF80620FFF7A1F807F50D7001F09D
S1132C78D4FB3470BDE8F0811448FFF7A1F8174C71
S1132C88D4F83C22D4F84002824259D12048FFF7B4
S1132C9897F8FFF7AAFA054600283BD10A48FFF738
S1132CA88FF80720FFF782F804F50D7001F0B5FBE3
S1132CB8014A1570BDE8F081580700204E5D0000F8
S1132CC8715D000098090020495E0000965D0000CF
S1132CD89B5D0000BF5D00005C07002064070020C6
S1132CE8BC0B0020ED5D000018070020F65D000015
S1132CF81A0700201C0700201E070020E95D0000B9
S1132D080F5E0000305E0000515E00005E5E000051
S1132D18755E00000B48FFF753F80B48FFF750F8AF
S1132D2804F50D7001F079FB0848FFF749F8084BE2
S1132D3800211970FFF71AF8BDE8F041FFF786B8CB
S1132D48BDE8F081965D0000915E0000A95E000078
S1132D585807002010B50023934203D0CC5CC45418
S1132D680133F9E710BD002310B50446184642089C
S1132D78E15C42EAC010013342180B2B02F0FF0059
S1132D88F5D110BD08B580B1036873B11A7862B182
S1132D98D9888088814208D15878FEF74DFD10F013
S1132DA8010F0CBF0020032008BD092008BDF8B599
S1132DB803690C4601F10902002B4DD04369114601
S1132DC81F7B00255E5D0A46202E13D0052E14BFF6
S1132DD83246E52207F00806F6B22EB1A2F1410602
S1132DE8192E01D82032D2B2013501F8012B082D51
S1132DF80A46E7D11E7A202E17D02E2201F8012B7D
S1132E0808269D5D0A46202D0FD007F01002D2B285
S1132E182AB1A5F14102192A01D82035EDB20136AB
S1132E2801F8015B0B2E0A46EBD1D97A21729E7FF9
S1132E38DD7F310441EA05661D7F597F2E4346EA4A
S1132E48012626605D7E197E41EA0526A680DD7D81
S1132E589B7D43EA0521E18000251570A669E6B14A
S1132E68E269D2B103690BB9002514E0018C4FF66D
S1132E78FF729142F8D0C76937F8150058B100219C
S1132E8801F040FC0028EFD0E369591E8D42EBD2D3
S1132E9870550135F0E700207055F8BDCA7E8B7E69
S1132EA8032843EA022305D1487D097D41EA00222B
S1132EB843EA02431846704710B504460A46407868
S1132EC804F134010123FEF7BFFC80BB94F83322DC
S1132ED894F8323243EA0221174B0AB29A4228D1B3
S1132EE894F86C2094F86D10130494F86A2043EA5B
S1132EF8016194F86B30114341EA03210F4B21F02F
S1132F087F429A4216D094F8880094F889100204F3
S1132F1894F8860042EA016194F88720014341EA63
S1132F28022121F07F40C01A18BF012010BD0320E0
S1132F3810BD022010BD00BF55AAFFFF4641540032
S1132F482DE9F041154602681378303B092B05D862
S1132F5854783A2C02D10232026000E000230020A7
S1132F680860002B40F05A81B54C2468002C00F00E
S1132F7858810C60217881B16078FEF75DFCC10747
S1132F880BD4002D00F0508100F00401C8B20028D1
S1132F9814BF0A200020BDE8F08100202070607072
S1132FA8FEF736FBC20700F142812DB100F004039D
S1132FB8DAB2002A40F03E8100212046FFF77CFF68
S1132FC8012818D194F8F60110B90D20BDE8F08154
S1132FD894F8FC5194F8FD112B0494F8FA0143EA8F
S1132FE8016294F8FB11024342EA0125204629466E
S1132FF8FFF762FF00E00025032800F01E81002887
S1133008E3D194F8402094F83F3043EA0220B0F525
S1133018007FDAD194F84B6094F84A1051EA0621FB
S11330280DD194F85A3094F85B2094F85810180489
S113303840EA026694F859200E4346EA022194F8BD
S11330484460E161731E012BE670BED894F84120F8
S1133058A270002AB9D0501E1042B6D194F8460086
S113306894F8453043EA002398B21B072081ACD179
S113307894F8487094F8473053EA07230DD194F82C
S1133088563094F857701B0443EA076394F8547055
S11330983B4394F8557043EA072394F8438094F823
S11330A8427057EA082890D006FB01FC08EB101779
S11330B86744BB4289D3DB1BB3FBF2F3002B84D0F8
S11330C840F6F576B34206D94FF6F57293428CBFB3
S11330D80326022600E00126023305EB08027F19C5
S11330E8032EA36125626262E76213D100287FF48C
S11330F86CAF94F8622094F86300120442EA006208
S113310894F86000024394F8610042EA0022A26243
S113311898000FE000283FF458AF0CEB0200022E91
S1133128A06201D1580005E003225A4303F00103C9
S113313803EB520000F2FF13B1EB532FFFF445AF3A
S113314800204FF0FF31032E2161E0605AD194F83A
S1133158652094F86430607143EA02216A18626158
S1133168607804F134010123FEF76EFB002849D18D
S113317894F8330294F8322242EA0023314819B20F
S113318881423FD194F8362094F83730110441EA4B
S1133198036094F8343094F83520184340EA022147
S11331A8294881422ED194F81A2294F81B3211042A
S11331B841EA036094F8183294F81922184340EA53
S11331C80221224881421DD194F8223294F8232204
S11331D8190441EA026094F8202294F82132104339
S11331E894F81E2240EA032194F81F021304E160B4
S11331F843EA006194F81C0294F81D22014341EA51
S113320802232361124926700888421C93B20020C5
S11332180B80E38020632071BDE8F0810B20BDE8BA
S1133228F0810C20BDE8F0812846BDE8F081032038
S1133238BDE8F0810A20BDE8F0810120BDE8F081F5
S1133248440F002055AAFFFF525261417272416136
S1133258400F0020F8B50446007908B3256B04F143
S11332683407607839462A460123FEF731FBB0B9A2
S1133278636A20719D4201D20020F8BDE269981862
S11332888542F9D2E678012EF6D9E16960786D189D
S11332982A4639460123FEF71BFB013EF3E70120CA
S11332A8F8BD38B50446FFF7D5FF0346002B50D1C7
S11332B82278032A45D16079002842D0236304F197
S11332C834010025CD540133B3F5007FF9D15223DD
S11332D884F8343084F835306123AA2084F83630F1
S11332E884F81B32236984F833027220552284F847
S11332F8180284F81902180C84F8322284F81E0281
S11333084122E06884F8372084F81A2284F81C32B1
S1133318C3F307221B0E84F81D2284F81F32C0F35E
S11333280722030C84F82002000E84F8212284F872
S1133338223284F82302626960780123FEF7C8FA0E
S11333486571002160780A46FEF724FB003018BF37
S1133358012038BD38B5036B044699420D460CD09C
S1133368FFF778FF58B9607804F134012A4601233D
S1133378FEF76AFA18B9256338BD002038BD012064
S113338838BD836902399A1E914204D28278C06A90
S113339802FB01007047002070470129F8B5044674
S11333A80D465DD9836999425AD20178022928D0F9
S11333B8032937D0012950D1426A05EB550602EB9F
S11333C85621FFF7C7FF002847D1636AF005013685
S11333D804EBD05703EB5621204697F83470FFF7D7
S11333E8B9FF002839D1F60504EBD65494F8341003
S11333F8EB0747EA012201D51009F8BD1005000DB5
S1133408F8BD426A02EB1521FFF7A4FF28BB2D067D
S1133418ED0D6119641991F8343094F8350043EAD4
S11334280020F8BD436A03EBD511FFF793FFA0B959
S11334386D06ED0D611991F8370091F83620343195
S113344803064978641943EA024294F8343042EA9C
S11334580120184320F07040F8BD4FF0FF30F8BD4C
S11334680120F8BD70B504460D46E1808168012944
S113347801D1022070BD03689A699142F9D271B9E9
S11334881878032801D1996A49B919890020A942F1
S1133498E060EED99B6A03EB1512226119E09E786D
S11334A83601B5420ED32068FFF777FF421C014668
S11334B818D00128DDD923689A699042D9D2AD1B66
S11334C8ADB2EEE7E1602068FFF75BFF00EB151192
S11334D82161206805F00F0500EB45113431616165
S11334E8002070BD012070BD0129F8B504460D46C1
S11334F8164672D9836999426FD2017802293AD063
S1133508032949D0012964D1426A05EB550702EB26
S11335185721FFF71FFF00285CD1F805C20D15F0ED
S11335280105F3B207D0A11891F8340000F00F0197
S113353841EA0313DBB2616A0120A2180137207142
S113354882F83430204601EB5721FFF703FF0028A7
S113355840D1FF05FA0D15B1C6F3071607E0A31805
S113356893F83410C6F3032621F00F073E43A71837
S113357887F834602EE0416A01EB1521FFF7EAFE73
S113358840BB2D06EB0DE21882F83460C6F307261B
S1133598154682F835601DE0426A02EBD511FFF743
S11335A8D9FEB8B96D06EB0DE11891F837200D4630
S11335B8130603F070421643C6F30723320C81F84E
S11335C83460360E81F8353081F8362081F837605A
S11335D800E0022001212171F8BD0220F8BDF8B5F0
S11335E805460F4631B9C6686EB18069864228BF60
S11335F8012609E0FFF7D1FE01283BD9AB699842BF
S113360839D33E4600E001263446A96901348C4288
S113361804D3012E01D80020F8BD022428462146EF
S1133628FFF7BBFE48B1431C02D14FF0FF30F8BD91
S113363801281FD0B442E8D1EDE7284621466FF0AF
S11336487042FFF751FF98B947B92A69EC60511CD9
S11336580CD0531E01202B61687107E028463946B7
S11336682246FFF741FF0028EFD001E02046F8BDCD
S11336780128DAD00120F8BD2DE9F843C6880446AC
S1133688701C86B20F4616B90420BDE8F883236976
S1133698002BF9D016F00F085AD1591C2161E168A2
S11336A8206819B90289B242EED951E08278531ED2
S11336B813EA16124CD1FFF770FE0128054602D80A
S11336C80220BDE8F883411C02D10120BDE8F8833B
S11336D8206881698D4235D3002FD5D0E168FFF782
S11336E87EFF054600283CD00128E9D0421CECD0D6
S11336F82068FFF7AFFD0028E7D12268343200279D
S113370817540130B0F5007FF9D1D4F80090294658
S11337184846FFF736FEC9F8300020688378BB4274
S11337280DD9012202712068FFF794FD0028CCD13D
S113373820680137036BFFB2591C0163EDE7016B85
S1133748CF1B0763E56020682946FFF71AFE20614E
S11337582068E68000EB4813343363610020BDE839
S1133768F8830720BDE8F8832DE9F84F4FF0FF09E7
S113377806464C4630683169FFF7ECFD8046002860
S113378840F0838075692F78002F78D0EA7AE52F86
S113379802F03F0369D002F00800C1B211B10F2B47
S11337A863D101E00F2B4AD1D6F81CB0BBF1000F4E
S11337B85CD007F04000C1B231B1F48895F80D909F
S11337C807F0BF07348401E0A7424ED16B7B4B4519
S11337D84BD12A780D2122F04000441E4C434FF06F
S11337E801084FF0000A2A4B1AF803106A18507897
S11337F86B5C43EA0020B8F1000F0BD000F09EFF89
S1133808FE2C804631D83BF8140000F097FF0134B1
S1133818804502E04FF6FF71884226D10AF1010A79
S1133828BAF10D0FDFD12A7802F04000C3B24BB3CE
S1133838B8F1000F26D03BF814401CB315E024B9A6
S11338482846FFF790FA81451FD04FF6FF7232845D
S1133858B269D37A13F0010307D1E85CD15C013370
S1133868884202D10B2BF8D10FE0FF243046002107
S1133878FFF702FF804600283FF47CAF05E04FF0D5
S1133888040802E0791ECCB2F0E74046BDE8F88FA0
S1133898625F00002DE9F74F0B7806462F2B894607
S11338A801D05C2B01D109F101090024B46099F815
S11338B800001F2800F2948030462146FFF7D2FD0D
S11338C874611FE15C2900F08B80D6F81CB00025D8
S11338D8785D6C1C1F2800F28B8007EB04091F28F5
S11338E894BF042400240BEB4500002D00F0048150
S11338F830F8021D202900F098802E2900F09580C8
S11339080023B2690BEB45072BF815302020D0545F
S113391801330B2BFAD14FF000083BF8181020297B
S113392800F085802E2900F08280B8F1000F01D0C4
S113393844F003043B4633F8027D2E2F01D0013DA9
S1133948F9D100224FF0080A17463BF8183008F15D
S11339580108002B6ED1B3691978E52901D1052036
S11339681870BAF1080F01D1BA00D7B207F00C03E6
S11339780C2B00F0A88007F00301032900F0A380B2
S113398804F00200C2B24AB907F00307012F08BFC6
S113399844F01004042B08BF44F00804B36930460B
S11339A8DC720021FFF75EFD10B93046FFF7DCFE3C
S11339B8B169CA7A002840F0898002F00403D9B2B8
S11339C8002940F09F807169C87A00F01002D3B2D0
S11339D8002B00F0858034682078FFF75FFAB06028
S11339E84F46397809F101092F297FF46BAFF7E7BE
S11339F82F283FF472AF5C283FF46FAFB4F5807F93
S1133A087AD0012100F07EFE002875D07F2806D8E0
S1133A183D4A12F8013F13B18342FAD16CE00BEB33
S1133A28440525F8020C254652E7013D5DE708F1F7
S1133A38010872E7202B03D02E2B04D1A8455DD0B2
S1133A4844F0030481E7524502D2A84515D155E054
S1133A58BAF10B0F04D144F003044FF00B0A7AE7D0
S1133A68A84503D044F003043FF675AFBF00FFB286
S1133A78A8464FF00B0A082267E77F2B0ED9184691
S1133A880021019200F03EFE019A034618B11F4836
S1133A98C11811F8803C44F002042BB11C4810F8FA
S1133AA8011F29B19942FAD144F003045F2306E0C7
S1133AB8A3F1410081B2192914D847F00207B0696B
S1133AC88354013241E744F0020459E7042819D128
S1133AD802F00401C8B2002814BF0420052011E034
S1133AE805200FE0A3F1610081B21929E7D8203B32
S1133AF847F001079BB2E2E7062003E0BAF10B0F97
S1133B08B4D1A8E7BDE8FE8FD15E0000E25E0000F4
S1133B18DA5E000038B5018CC5884FF6FF73994208
S1133B2808BF29460446FFF79DFC0146B8B9216938
S1133B382068FFF70FFC014670B96069E52202703E
S1133B48236801201871E288AA4208D22046FFF7A8
S1133B5893FD01460028EAD0042908BF022108463B
S1133B6838BD00002DE9F041FF2704463D460426F0
S1133B782169002967D02068FFF7ECFB0646002876
S1133B8862D163691A78002A64D0E52AD97A51D0B7
S1133B982E2A4FD001F03F0008284BD00F283FD1E0
S1133BA802F04006F1B229B1E5885F7B02F0BF025A
S1133BB8258401E0AA423DD1587BB8423AD119780C
S1133BC80D2001F03F05691EE66941434FF0010EDF
S1133BD80020234D10F805C003EB0C0595F801806F
S1133BE813F80C5045EA0825BEF1000F06D0FE294B
S1133BF820D826F81150AE46013103E04FF6FF7C79
S1133C08654517D101300D28E3D11B7803F0400531
S1133C18E8B2E0B1FE290DD8002326F8113016E0E9
S1133C2825B91846FFF79FF8874215D04FF6FF735A
S1133C38238411E0FF2520460021FFF71DFD0646D9
S1133C48002895D000E03EB10021216104E0013A4A
S1133C58D5B2F0E70426F7E73046BDE8F08100BFA7
S1133C68625F0000012970B504460D4622D98369B4
S1133C7899421FD2A069854205D220462946FFF7FA
S1133C888CFB064608B9002070BD012812D0431CDD
S1133C980ED0204629460022FFF726FC58B9216990
S1133CA8481C03D04A1C0125226165713546E1E7A9
S1133CB8012070BD022070BD73B51C4616460B2248
S1133CC80546FFF747F8052C0AD9B21E32F8020F49
S1133CD8630843EAC434538821188CB2002BF5D105
S1133CE8072304F00F0000F13002392A88BF00F1DD
S1133CF837020DF80320013B2409F2D102A9C818A0
S1133D087E2200F8082C9C4204D0295D202901D089
S1133D180134F8E7072B05D802AAD11811F8080CC2
S1133D28013300E0202028550134072CF2D97CBD4A
S1133D382DE9FF418669D0F81C800C2204463146DF
S1133D4801A8FFF707F89DF80F30DA0722D50020FD
S1133D58F0720127E061304601A942463B46FFF76D
S1133D68ABFF20460021FFF77DFB054650B92046EE
S1133D78FFF7FAFC054628B90137BFB2642FEAD128
S1133D880725B2E0042D40F0B0809DF80F10F172C1
S1133D98C4F81C809DF80F2002F00205EBB20BB9A1
S1133DA801270CE0002038F8107017B1471CB8B28E
S1133DB8F9E700F119010D2291FBF2F5AFB22046A3
S1133DC80021FFF74FFB0546002840F08E80064689
S1133DD820682169FFF7BEFA0546002840F085806F
S1133DE863691878E52800D018B90136BE4201D1B4
S1133DF808E02E4620460121FFF73EFC0546002830
S1133E08E6D072E0013EB6B2002E53D0E1882046D7
S1133E188A1B91B2FFF726FB0546002865D1A069E5
S1133E28FEF7A1FF074620682169FFF793FA0346C6
S1133E380546002859D162690F20F5B2D4F81CE070
S1133E48691ED0720D204143577313739376D3764A
S1133E5818464FF6FF7CDFF89C80634518BF3EF890
S1133E68113010F808C04FEA132802F80C309444B3
S1133E7818BF01318CF8018001304FF6FF7C002B0C
S1133E8808BF63460D28E4D1634502D03EF81130DB
S1133E9813B946F04005EDB21570216801220A7184
S1133EA820460021FFF7E8FB0546F0B9013EB6B20B
S1133EB8002EB8D120682169FFF74CFA0546A0B94D
S1133EC860692B460021C1540133202BFAD1606963
S1133ED8A1690B22FEF73EFFA2696069D17A01222B
S1133EE801F01803037320680271284604B0BDE882
S1133EF8F08100BF625F000048B9064A136803B145
S1133F08187009B1002008701160002070470B2058
S1133F18704700BF440F00202DE9F0478EB001918F
S1133F2816460546002800F098800023036005A97A
S1133F3801A802F01E02FFF703F88046002840F0AB
S1133F4895804C4902A80B900C9105A80199FFF79C
S1133F58A1FC0A9C18B9002C0CBF0620002016F0FE
S1133F681C0F06F01F0748D048B1042802D105A841
S1133F78FFF7DEFE47F008070A9C48B175E0E17ACE
S1133F8811F0110F70D106F00403DEB2002E67D1D0
S1133F9807F00802D0B200283DD0FDF7F9FDC0F3C0
S1133FA80726E673010C0026030EDDF8149021742D
S1133FB8E67226776677A677E677A073637499F82E
S1133FC800002146FEF76AFF0122A676E6762675EA
S1133FD8667589F804200646E8B148463146D9F89A
S1133FE830A0FFF73FFE00283FD10598013EC66088
S1133FF85146FFF7AFF970B137E0002835D1E37ABD
S113400803F01002D0B200282CD106F00206F6B252
S11340180EB1D90728D407F00800C1B209B147F096
S11340282007059E2146336B2C62EB61AF71307813
S1134038FEF734FF2861A07FE27F010441EA0263AE
S1134048227F607F1343F28843EA00210023E9605A
S1134058AB60AB612E60AA8008E04FF0090805E068
S1134068082002E0042000E00720804640460EB005
S1134078BDE8F087400D00202DE9F74F9A4600234C
S1134088CAF80030044688461746FEF77BFE054604
S1134098002840F0A080A179080600F19980C9079A
S11340A840F19880E068A268861AB74238BF3E4655
S11340B8002E00F09080A168CB0570D12068837829
S11340C85A1E02EA512313F0FF030CD109B92069DF
S11340D804E061690193FFF760F9019B01280BD99A
S11340E8421C55D06061D4F800B061695846019308
S11340F8FFF747F9019B20B9A07960F07F03A3710A
S113410866E05FEA562900EB030724D09BF80220F7
S113411809EB0300904288BFC3EB020941469BF8B0
S113412801003A465FFA89F3FDF78EFBA17980BB5B
S113413801F04001CBB25BB1A269D71B4F4507D24E
S113414808EB472004F124014FF40072FEF702FE45
S11341584FEA492731E0A269BA421FD0A07900F09A
S11341684001CBB25BB104F124019BF801000123A7
S1134178FDF7AEFBA17960B921F04002A271214696
S113418851F8240B3A4640780123FDF75DFB28B12A
S1134198A17961F07F05A57101251CE0A761A768D5
S11341A84046F905CB0DC3F50077BE4238BF374604
S11341B8E11824313A46FEF7CDFDA068DAF800305C
S11341C8C119DA19A160B844CAF80020F61B6FE7D0
S11341D8022500E007252846BDE8FE8F2DE9F74FA4
S11341E899460023C9F80030044688461746FEF766
S11341F8C9FD0546002840F0B780A079010657D4C8
S113420800F00201CAB2002A00F0AD80E368DF4280
S113421828BF002730E05FEA572B00EB0A0674D06A
S113422898780BEB0A01814288BFCAEB000B414620
S1134238587832465FFA8BF3FDF74AFB002873D1AE
S1134248A3699E1B5E450BD204F124004FF400724F
S113425808EB4621FEF77EFDA27922F04000A0710A
S11342684FEA4B26A168D9F800208B199019A3604E
S1134278B044C9F80000BF1B0FB3A168CA055AD1DE
S1134288206890F802A00AF1FF3202EA512313F0E1
S1134298FF0A1DD171B9216921B9FFF7A0F90146B7
S11342A8206161B10129A3790FD163F07F01A17164
S11342B8022559E06169FFF792F90146F1E7A06820
S11342C8E26890424AD9E06048E04A1C2DD0616116
S11342D8A07900F04001CAB262B1214651F8243BEA
S11342E8A26958780123FDF7F3FAA379E8B923F012
S11342F84000A0712268616910460192FFF741F8F5
S1134308019B002887D1A379CFE7A169B14211D0D5
S1134318A068E26890420DD2587804F1240132462C
S11343280123FDF791FA28B1A37963F07F05A571FC
S1134338012519E0A661A668F305D90DC1F5007633
S11343486018B74238BF3E46243032464146FEF72D
S113435801FDA07940F04002A27183E7A37943F0FC
S11343682001A17100E007252846BDE8FE8F70B53D
S11343780446FEF707FD00284ED1A37903F0200276
S1134388D1B2002948D003F04000C3B26BB1214632
S113439851F8242B01235078A269FDF799FA0028D3
S11343A839D1A67926F04001A1712068E169FEF7A8
S11343B8D1FF0646002E2FD1256AE87A40F0200363
S11343C8EB72E2682A77A189080A6877E389AB77F0
S11343D8E27BEA7721690B0C1A0AC1F30720A97654
S11343E82B756A75E876FDF7D3FBA875030CC0F343
S11343F80721000EE97568762B76AE74EE74A279FF
S11344082368012022F02001A17118712068BDE8F9
S11344187040FEF746BF012070BD10B50446FFF793
S1134428A6FF00B9206010BDF8B504460D46FEF796
S1134438A9FC0646002840F09380A279110600F1F1
S11344488E80E3689D4205D902F00200C1B20029BA
S113445808BF1D460022A368A2600DB900254DE0DF
S1134468206887787F026BB1013B691EB1FBF7F1C5
S1134478B3FBF7F2914205D378420340A360ED1AE7
S113448861690AE0216939B9FFF7A9F801280146E9
S11344982DD0431C52D0206161610029DED0BD4279
S11344A81CD9A379206803F00202D3B223B1FFF721
S11344B896F8014618B910E0FEF76FFF0146481C4C
S11344C83CD0012913D92068826991420FD2A3688C
S11344D86161D819A060ED1BE1E73D46A268531954
S11344E8A360EB05BAD02068FEF74BFF20B9A0798A
S11344F860F07F02A27132E000EB5525A168CB057C
S113450823D0A269954220D0A07900F04003D9B203
S113451859B1214651F8240B01234078FDF7D8F905
S1134528A17960B921F04002A271214651F8243BD7
S11345382A4658780123FDF787F928B1A17961F053
S11345487F06A67101260BE0A561A168E068814297
S113455806D9A279E16042F02003A37100E00226A3
S11345683046F8BD30B58FB00EAB43F8340D0D4668
S1134578184605A90022FEF7E3FC044688B90A494F
S113458802A80B900C9105A80199FFF783F904463A
S113459838B90A9A22B105A82946FEF708FC00E0B2
S11345A8062420460FB030BD400D002070B598B0E9
S11345B818AB43F85C0D184606A90122FEF7C0FCA7
S11345C8044600284DD1284903A80C900D9106A84B
S11345D80199FFF75FF90446002842D10B9E36B1D2
S11345E8F27A12F0010F0CBF0024072400E006241D
S11345F8069D31462878FEF751FC0546002C30D13B
S1134608F47A04F01003D8B2C8B1012D13D90FA855
S113461806A92422FEF79EFB0FA802211195FEF796
S113462821FF0446E8B90FA8FFF79CFA044620B115
S1134638042804D015E0022413E0072411E006A896
S1134648FFF768FA044660B925B90698FEF729FE0B
S1134658044606E006982946FFF704FB04460028AA
S1134668F3D0204618B070BD400D00202DE9F34169
S113467806460F469046054600247B1E9C4211DAE6
S113468801224046694601ABFFF7F6FC0198012870
S113469808D19DF800100D29EFD001340A2905F836
S11346A8011BEAD100222A70944214BF30461046F6
S11346B8BDE8FC810A2837B504460D4602D10D2011
S11346C8FFF7F8FF02A901F8084D284669460122B8
S11346D801ABFFF783FD0198012814BF4FF0FF30A9
S11346E801203EBD70B505460E460024285D38B14C
S11346F83146FFF7DFFF431C01D00134F6E70446D7
S1134708204670BD7F2816D931B1FF2812D80A492E
S1134718803831F810007047074A8BB232F81120FC
S1134728824203D001318029F6D10B4603F180007F
S1134738C0B2704700207047506100000023064A49
S113474832F8131031B1884201D00133F7E7034836
S113475830F81300704700BF705F0000506200001B
S113476810B5013A8A1891420CD20C784B7803EBB5
S113477804239BB2181880B2984201D2431C98B201
S11347880231F0E707D10B781902081880B2884281
S113479801D2421C90B210BD38B50E4C0822657C7B
S11347A8237C143D05EB03218DB2401904F11A0151
S11347B880B2FFF7D5FF04F122012A46FFF7D0FFA4
S11347C820B1020A42EA002398B238BD4FF6FF70BE
S11347D838BD00BFC20F002070B5C478124B0A1947
S11347E8D4B2DC7085780E0A7219D2B29A70457800
S11347F8B2425D700078187005D20135EDB25D7073
S11348080DB901301870C9B28C420CDA531C064831
S1134818DAB282703AB941784B1CDAB2427012B9F2
S113482801784B1C037070BD1116002010B5084C9C
S1134838014620680830FFF7CFFF064A236811783D
S1134848507819729178D27858729972DA7210BDC8
S1134858480F00201116002008B50020064914222C
S1134868FFF77EFF20B1030A43EA002080B208BDA7
S11348784FF6FF7008BD00BFD00F00200620FFF7D9
S11348888BBF0000064900231A460B80054B012004
S11348980549187005484A764FF4806202807047CB
S11348A822160020201600204C0F00201616002087
S11348B8044A054B118811B91970108070470120FA
S11348C8187070472216002020160020F8B5834B74
S11348D883491C68834B032803F136020A60824922
S11348E80A600AD1607E00F00F03032B40F0BE84F7
S11348F8218A002940F0BA846DE002286FD17B48F0
S1134908C278511CCBB2C37063B98278511CCBB244
S113491883703BB94278511CCBB2437013B9027807
S1134928511C0170724B734A002018801080607EFD
S1134938072801D005280AD1A07E431CD9B27829BA
S1134948A17640F093840022627600F08FBC0028A0
S113495800F08C84218A002938D0A27E511EA176C9
S1134968002A40F08384E37E082B04D0421E012AE7
S113497809D8052B07D100235F4A8021637611707B
S113498800F0D6FE60E3042B04D8032202FA03F2F3
S1134998D1B200E0302100F00F00A1760133411EAE
S11349A8E376072900F26284DFE811F08001080049
S11349B80A00EC026004EC026004EC02002576E1D3
S11349C84D4B04221A7000F0B3FE5CE300F00F03B1
S11349D8032B40F04B844848082202709DE2987BE0
S11349E8452840F0438442481E7C5A7C018802EBE7
S11349F806268E4200F33A841A7DB6B292060680E1
S1134A0840F034845B7D002B40F030843B480488BC
S1134A180CB9418849B1334AD38BA34240F0268468
S1134A28118C4088814240F02184FFF715FF4FF62E
S1134A38FF729042074640F019842A4DEB7D062BFD
S1134A481DD0012B40F0128495F82210082940F05B
S1134A580D84AB8C4FF6F6720020934285F8220041
S1134A6801D9093300E008331E49AB84488B234A33
S1134A788B8BC88350880B844C838883DFE3FFF7D0
S1134A88FDFEB84240F0F2831D4B5C7E84B1A98CD4
S1134A989A8891420CD1688CD988884208D1688B4D
S1134AA81A88904204D1A98B5888814200F01A814F
S1134AB80C4B93F82F2002F03F0102292AD19A8C3B
S1134AC81048114602801048104B008882421FD1BA
S1134AD8002C74D100241C70094C7AE0480F002083
S1134AE804160020C20F00202416002008160020F7
S1134AF8B80F0020C00F0020101600200C1600204C
S1134B084C0F002018160020221600202016002022
S1134B1801221A707B4B93F82F1001F00400C2B2E3
S1134B28002A40F0A38393F82D20774914252824DC
S1134B380C8083F82F5093F8294093F82C5083F86D
S1134B48292093F82B20502093F8271083F82E005F
S1134B5883F8272093F8280093F8262083F8285010
S1134B686A4D01342A7093F82A5083F82C0083F88C
S1134B782650E5B283F82B1083F82A2083F82D50A9
S1134B8865B90130C4B283F82C403CB90131CDB2C7
S1134B9883F82B5015B9013283F82A20594B5C4C01
S1134BA8588C5D8B2080998C98845A4859849A8BA8
S1134BB804884188DD831A845C83998317E3564803
S1134BC80122072C0CBF044600241A70002C00F0A4
S1134BD84D83524D0326A6762676042300262C60A0
S1134BE8484DE375A675E676A18095F8221095F8E8
S1134BF823006B8B41EA0022E280A98B484A238078
S1134C0861801378517823736173937895F8291028
S1134C18D278A373E27395F8283095F82720E172C7
S1134C2895F82610012060762082A37262722172A0
S1134C38FFF7FCFD95F82E5005F0F000502835DDFF
S1134C482B0938495A1F95000A783346AB4229DAAA
S1134C582C48C11891F8362022B3012A01D1013316
S1134C681EE0022A17D191F83760042E13D12D487B
S1134C78264D027091F8382091F839102B70244D84
S1134C8841EA022340F20A602B80834228BF03468C
S1134C986382A3820AE0C01890F8371011B1CB18C8
S1134CA8DBB2D3E719491F4D0B702A70102515483C
S1134CB8144B80F82F5093F82F10042041F002026F
S1134CC8022583F837001048062183F82F2083F83B
S1134CD836500A222C2583F8381083F839200580A9
S1134CE860214AE20D4F95F82F203B600E4902F0EF
S1134CF804070020FFB20870C7B1587620230B7050
S1134D08E8E100BFC20F0020B80F002020160020E1
S1134D18181600200C1600204C0F0020480F002005
S1134D2808160020281600201016002095F82E30AA
S1134D38143E19098800964B361A964904F00F0454
S1134D48B6B2022C18700E8003D102F03F0012286C
S1134D580ED00EB994070BD08F49904BCC8C188980
S1134D68844240F00082098D5B89994240F0FB81BE
S1134D7802F01002D4B2002C44D0884C218A0029B5
S1134D8840D004F10C00FFF727FD834A844B92F8C6
S1134D982A001D78854235D192F82B10587888421C
S1134DA830D192F82C609978B1422BD192F82D2009
S1134DB8DB78934226D16073E07E2573A173E37395
S1134DC8C0B9227EA37EA17DD01AA0EBD102D3B2B2
S1134DD8DAB25918C9B21006A17501D55C42E2B21B
S1134DE86E4BD87DA0EB9004A218D0B200EBD10191
S1134DF8D875197669486B4B027E012400211C7012
S1134E0882760182654B674A597E01F00F04601E61
S1134E18072800F22B82DFE810F008001D008D003F
S1134E28600181019D01A601540111785D4CCA07F6
S1134E3840F11C820320002158761982554B4022E8
S1134E4818882270002800F0EF8042222270FFF7B1
S1134E58EDFCE9E01478E30762D54F4B93F82F2073
S1134E6802F03F0012285BD193F82E3003F0F002D1
S1134E78502A36DD4C491809441F0A78A400002337
S1134E88A3422ADA4448C11891F836202AB3012AE1
S1134E9801D101331FE0022A18D191F83750042DAB
S1134EA814D141483A4C027091F8382091F83910DD
S1134EB823703E4B41EA022440F20A60374A1C80C0
S1134EC8844228BF0446548294820AE0C01890F8A9
S1134ED8371011B1CB18DBB2D2E72D49324C0B7025
S1134EE822702E4C2C4B032093F8262093F827107D
S1134EF8607693F8280093F8293022726172A072C0
S1134F08E3720120FFF792FC264942220A70214BE2
S1134F18274A002020821880108000F009FC89E0CC
S1134F28204C2021217000F003FC224B0022186839
S1134F384276EFE5184C94F82F30D8073CD501F0A9
S1134F481002D0B2002837D11448018A002940F051
S1134F588D81104D2A88541CA0B2FFF767FC114BB1
S1134F682D88187840F01001197015B140F012021C
S1134F781A700A4C00F0DCFB01230820002123826C
S1134F886076E1761122044D85F82F20F0E000BF09
S1134F9820160020B80F0020C20F00204C0F00205C
S1134FA811160020101600202816002018160020BC
S1134FB8C00F0020480F002003F02004E3B273B1AF
S1134FC8A04AA14B92F8340092F8354044EA0022F2
S1134FD8186884181C609D4B1888821A1A809B4C88
S1134FE8208850B101F01001CBB233B9984C227823
S1134FF842F002012170FFF719FC924890F8304002
S113500890F83130934803EB0422818A94B2924B8E
S11350188C421C8000D804B919808D4C1A882378D6
S113502842829A0700F022818C480024048000F010
S11350387FFB884C864B894A1B7803F02001C9B250
S113504821B100231380637614229CE703F0100037
S1135058C0B230B101250420118025826076E17642
S113506890E7118869B1DB0748BF2082228A7B4B0D
S113507832B9608A814288BF18801988218200E089
S11350881A800022E276764B744A18686E491388AF
S1135098086033B1208A20B16C4B2830188018225C
S11350A80BE06B490A7802F00203D8B2002800F03A
S11350B8DD806648282505801022624981F82F2062
S11350C859E01178CA0740F1D18000245C76604B1E
S11350D81020187000F02CFBC8E05C48008808B168
S11350E8FFF7A4FB574B5A4993F82F20087812F07E
S11350F801040CD010F0010F564D05D000220723EF
S11351086B76AA762A8218E006246C7615E0C00726
S11351181CD55048052141760482A7E04B480088F5
S113512808B1FFF783FB474B93F82F20D1070DD520
S1135138484D072100246976AC760120FFF776FBF9
S113514843491020087000F0F3FA0CE03F4B1A882A
S11351584AB98BE01278D20740F1888007210024ED
S113516859769C7682E0374910253A4C81F82F50BD
S1135178364B28201880334B502183F82E10227A7E
S1135188304D85F82A20607A85F82B00A17A85F8B5
S11351982C10E37A85F82D30227B85F82620607B55
S11351A8062285F82700A17B85F82810E37BEA7599
S11351B885F82930A0882B4B6884E188A98418884D
S11351C859886883A9832388EB8360882884647E4C
S11351D804F01001CBB22BB1002085F8310085F81A
S11351E8300004E085F830200A2285F83120174978
S11351F8144C0B8840251A0AA5750025227463747B
S113520884F8355084F8345084F8325084F8335094
S1135218FFF734FB144AC043608613884521581CA1
S1135228A17381B211800A0AE57365752575A274A4
S1135238E17425766576FFF70FFBC34323830022C9
S113524818E000BFC20F002004160020B80F002089
S1135258101600204C0F002018160020C00F002044
S1135268241600200C160020BA0F0020034900233E
S11352781A460B8002480270F8BD00BFB80F002020
S113528810160020030A43EA002080B27047000089
S11352980A1E034609DD0548054900680A80834259
S11352A803D0194692B200F087BA7047241600203A
S11352B8C00F002038B52C4B988BDD8B0023072BAF
S11352C811D80C225A4329498C18895A41B1628849
S11352D832B1884204D1954202D12548037039E09D
S11352E80133DBB2EBE70023072B0DD80C2058431E
S11352F81E490A5A0C1822B9618811B91C4803704E
S113530823E00133DBB2EFE7194A082B13701CD1F1
S113531818480023057819461A46072A13480BD853
S11353280C2404FB0200847A281B9842C4BFC3B22D
S113533811460132D2B2F0E70F4C0D4A23700C2407
S113534804FB01040D4B1170197020460C4904220A
S113535800F032FA0B490622201D00F02DFA054907
S11353680A78A27238BD00BFC20F00202C16002094
S1135378291600208D1600202A1600208C160020DD
S1135388DE0F0020D80F002008B5124B00211A7830
S1135398501C1870104801700F490B78072B17D848
S11353A80C2043430D4AD0184188D35A41EA0302DA
S11353B891B249B1074B817A1A78531A772B03DDD6
S11353C80021042200F006FA03480278511CE2E79F
S11353D808BD00BF8D160020291600202C160020B9
S11353E8F8B52A4D2B88292B4FF000033DD9284CBA
S11353F81F46A08A2B80B0F5807F03D0B0F5007FCC
S113540842D134E0234EE18C328891423CD1208D44
S11354187388984238D1FFF74DFF0221617506223F
S113542804F1160104F12000277500F0C5F91A49A2
S1135438062204F1160000F0BFF917490622A01D40
S113544800F0BAF904F120010622204600F0B4F96C
S1135458A28BE08B33887188E28420850822062099
S1135468A383E183227360732A232B80F8BD094B3D
S1135478E18C1A88914207D1208D5B88984203D128
S1135488BDE8F840FFF716BFF8BD00BFB80F00200D
S1135498C20F00200C1600201A160020434838B505
S11354A8C38B4FF6FF72934204D1028C9A4201D106
S11354B83F4968E03F4C404A258810885D400542D2
S11354C807D13A4D6488288C528880EA040515422D
S11354D806D03A4D3A4B28886A8818805A8002E0E8
S11354E8374C23806080364C002520886488072D3B
S11354F80CD80C236B43334AD118D25A824202D1B6
S11355084B88A3423BD00135EDB2F0E72E4B082D72
S11355181D7036D1254CFF212046062200F05AF989
S113552804F120000021062200F054F9A01D2749A7
S1135538062200F041F904F116002449062200F07D
S11355483BF91F491B4B08884A88E0841988588806
S113555800232375A37363742285A183E083062142
S1135568012204201A4B61736275E2732574A174D5
S1135578E074257336341C602A21164813E0124857
S113558805700A480431062200F016F90F4906226C
S1135598114800F011F90549082200230D480A733F
S11355A84B7301880E31018038BD00BFC20F002043
S11355B8306400000C160020B40F0020BC0F00203B
S11355C88E1600202C160020291600201A160020FA
S11355D804160020B80F0020C80F002008B5FCF7F7
S11355E8DBFAFCF72FFE134B00F5FA701860FCF792
S11355F829FE114A00F51C5110311160FFF742F9D8
S11356080E484FF6A96243F61373028043800C4890
S11356184FF6FF710023018043800A48028040F25C
S1135628131242804EF60300FFF742F9BDE8084022
S1135638FCF7BEBA98160020941600200C16002019
S1135648B40F0020BC0F002038B50C4B1C68002395
S1135658E26922629AB28A4205D2C55CE21882F8EB
S113566824500133F6E70431A4F8641004F120004F
S1135678FFF70EFEE069411CE16138BD480F0020C8
S113568870B5FCF71BFB00B3234C244D20804FF46A
S11356980060AE89FFF7F6FD864207D10120FFF7C7
S11356A815F9208888B1FFF7F9FE0AE040F60600EC
S11356B8AD89FFF7E7FD854207D1FFF791FE2388FF
S11356C81BB1FCF715FB00212180FCF7BBFD144B33
S11356D81A68904211D302F5FA74124812491C60F0
S11356E80D4C08600220FFF7F1F823882BB1FFF76F
S11356F8D5FEFCF7FDFA00222280FCF7A3FD0B4936
S11357080B68984205D303F51C5010300860FFF766
S11357183BFE002070BD00BFB80F0020C20F002060
S1135728981600204C0F0020480F002094160020E3
S113573810B5174B17481C68037803F04002D0B221
S113574828B101230022E361A4F8642010BDD9071D
S113575803F00401CBB248BFA4F8640033B1B4F831
S1135768641019B104F12000FFF792FD094A10787A
S113577800F00201CBB24BB1074800220168A4F83B
S11357886420081DBDE81040FCF7D4BE10BD00BF5E
S1135798480F00201016002004160020303809286D
S11357A88CBF002001207047A0F16103D9B21929E8
S11357B898BF2038704700004FF00003002A07D034
S11357C811F803C000F803C003F10103013AF7D14B
S11357D8704700BF0346002A00F0048003F8011B49
S10B57E8013AFBD1704700BF38
S11357F040420F0000201C0080841E000080250011
S1135800999E36000040380000093D0000803E00AB
S113581000004B00404B4C0000204E00808D5B008C
S113582000C05D000080700000127A0000007D005E
S113583080969800001BB7000080BB00C0E8CE0033
S1135840647ADA000024F4000000FA0080A812014F
S1135850002D310100366E0140787D01433A2F5707
S11358606F726B2F736F6674776172652F4F7065FB
S11358706E424C542F5461726765742F44656D6F8A
S11358802F41524D434D335F4C4D33535F454B5F76
S11358904C4D3353363936355F43726F7373776FBC
S11358A0726B732F426F6F742F6964652F2E2E2FC6
S11358B06C69622F6472697665726C69622F7379A0
S11358C07363746C2E63000000E10F4004E10F4029
S11358D008E10F4040E00F4044E00F4048E00F4033
S11358E0433A2F576F726B2F736F667477617265CB
S11358F02F4F70656E424C542F5461726765742F3C
S113590044656D6F2F41524D434D335F4C4D3353BE
S11359105F454B5F4C4D3353363936355F43726FB9
S11359207373776F726B732F426F6F742F69646533
S11359302F2E2E2F6C69622F6472697665726C69E2
S1135940622F6770696F2E6300433A2F576F726B33
S11359502F736F6674776172652F4F70656E424C5A
S1135960542F5461726765742F44656D6F2F4152D3
S11359704D434D335F4C4D33535F454B5F4C4D337B
S113598053363936355F43726F7373776F726B7347
S11359902F426F6F742F6964652F2E2E2F6C6962EE
S11359A02F6472697665726C69622F666C617368C4
S11359B06C69622E6300433A2F576F726B2F736FBB
S11359C06674776172652F4F70656E424C542F5424
S11359D061726765742F44656D6F2F41524D434D5D
S11359E0335F4C4D33535F454B5F4C4D3353363926
S11359F036355F43726F7373776F726B732F426FB9
S1135A006F742F6964652F2E2E2F6C69622F647258
S1135A10697665726C69622F756172746C69622E45
S1135A206300433A2F576F726B2F736F66747761FD
S1135A3072652F4F70656E424C542F5461726765C6
S1135A40742F44656D6F2F41524D434D335F4C4D60
S1135A5033535F454B5F4C4D3353363936355F43D3
S1135A60726F7373776F726B732F426F6F742F69DA
S1135A7064652F2E2E2F6C69622F647269766572AD
S1135A806C69622F7373692E6300433A2F576F72E8
S1135A906B2F736F6674776172652F4F70656E42FA
S1135AA04C542F5461726765742F44656D6F2F4198
S1135AB0524D434D335F4C4D33535F454B5F4C4D1B
S1135AC03353363936355F43726F7373776F726B46
S1135AD0732F426F6F742F6964652F2E2E2F6C699C
S1135AE0622F6472697665726C69622F6574686589
S1135AF0726E65742E63002F64656D6F70726F67CC
S1135B005F656B5F6C6D3373363936352E73726532
S1135B1063002F626F6F746C6F672E747874004328
S1135B203A2F576F726B2F736F6674776172652F9C
S1135B304F70656E424C542F5461726765742F44E4
S1135B40656D6F2F41524D434D335F4C4D33535F61
S1135B50454B5F4C4D3353363936355F43726F7363
S1135B6073776F726B732F426F6F742F6964652F35
S1135B702E2E2F2E2E2F2E2E2F2E2E2F536F75724C
S1135B8063652F41524D434D335F4C4D33532F4387
S1135B90726F7373776F726B732F766563746F7242
S1135BA0732E630000800000002000000400000049
S1135BB000A00000002000000500000000C000005C
S1135BC0002000000600000000E0000000200000AB
S1135BD00700000000000100002000000800000091
S1135BE00020010000200000090000000040010026
S1135BF0002000000A0000000060010000200000F6
S1135C000B00000000800100002000000C000000D8
S1135C1000A00100002000000D00000000C00100F1
S1135C20002000000E00000000E001000020000041
S1135C300F000000000002000080000010000000BF
S1135C40008002000080000011000000000003003A
S1135C5000800000120000000080030000800000AB
S1135C6013000000433A2F576F726B2F736F6674E3
S1135C70776172652F4F70656E424C542F54617278
S1135C806765742F44656D6F2F41524D434D335FEB
S1135C904C4D33535F454B5F4C4D3353363936359A
S1135CA05F43726F7373776F726B732F426F6F748E
S1135CB02F6964652F2E2E2F2E2E2F2E2E2F2E2E53
S1135CC02F536F757263652F41524D434D335F4CB3
S1135CD04D33532F756172742E63004F70656E429D
S1135CE04C5400433A2F576F726B2F736F6674775F
S1135CF06172652F4F70656E424C542F5461726708
S1135D0065742F44656D6F2F41524D434D335F4C85
S1135D104D33535F454B5F4C4D3353363936355F06
S1135D2043726F7373776F726B732F426F6F742F3D
S1135D306964652F2E2E2F2E2E2F2E2E2F2E2E2FD2
S1135D40536F757263652F66696C652E63004669CF
S1135D50726D776172652075706461746520726517
S1135D6071756573742064657465637465640A0D84
S1135D70004F70656E696E67206669726D77617237
S1135D80652066696C6520666F722072656164695E
S1135D906E672E2E2E004F4B0A0D005374617274E1
S1135DA0696E67207468652070726F6772616D6DCB
S1135DB0696E672073657175656E63650A0D0050C1
S1135DC0617273696E67206669726D7761726520AE
S1135DD066696C6520746F206F627461696E2065FA
S1135DE0726173652073697A652E2E2E0045726187
S1135DF073696E6720002062797465732066726F20
S1135E006D206D656D6F7279206174203078005259
S1135E10656164696E67206C696E652066726F6D7A
S1135E202066696C652E2E2E4552524F520A0D0083
S1135E30496E76616C696420636865636B73756D24
S1135E4020666F756E642E2E2E4552524F520A0DE7
S1135E500050726F6772616D6D696E672000206219
S1135E607974657320746F206D656D6F727920612C
S1135E70742030780057726974696E672070726F8D
S1135E806772616D20636865636B73756D2E2E2E6A
S1135E9000436C6F73696E67206669726D77617217
S1135EA0652066696C650A0D004669726D776172DA
S1135EB065207570646174652073756363657373BD
S1135EC066756C6C7920636F6D706C657465640ABB
S1135ED00D00222A3A3C3E3F7C7F002B2C3B3D5B4D
S1135EE05D00809A90418E418F80454545494949DE
S1135EF08E8F9092924F994F555559999A9B9C9D8C
S1135F009E9F41494F55A5A5A6A7A8A9AAABAC2118
S1135F10AEAFB0B1B2B3B4B5B6B7B8B9BABBBCBD25
S1135F20BEBFC0C1C2C3C4C5C6C7C8C9CACBCCCD15
S1135F30CECFD0D1D2D3D4D5D6D7D8D9DADBDCDD05
S1135F40DEDFE0E1E2E3E4E5E6E7E8E9EAEBECEDF5
S1135F50EEEFF0F1F2F3F4F5F6F7F8F9FAFBFCFDE5
S1135F60FEFF01030507090E10121416181C1E006B
S1135F7061006200630064006500660067006800F9
S1135F8069006A006B006C006D006E006F007000A9
S1135F907100720073007400750076007700780059
S1135FA079007A00A100A200A300A500AC00AF0014
S1135FB0E000E100E200E300E400E500E600E700C1
S1135FC0E800E900EA00EB00EC00ED00EE00EF0071
S1135FD0F000F100F200F300F400F500F600F80020
S1135FE0F900FA00FB00FC00FD00FE00FF000101C7
S1135FF003010501070109010B010D010F01110145
S113600013011501170119011B011D011F012101B4
S113601023012501270129012B012D012F01310124
S11360203301350137013A013C013E01400142018F
S11360304401460148014B014D014F0151015301F7
S11360405501570159015B015D015F016101630164
S11360506501670169016B016D016F0171017301D4
S1136060750177017A017C017E019201B103B203CB
S1136070B303B403B503B603B703B803B903BA0350
S1136080BB03BC03BD03BE03BF03C003C103C303FF
S1136090C403C503C603C703C803C903CA03300442
S11360A03104320433043404350436043704380428
S11360B039043A043B043C043D043E043F044004D8
S11360C04104420443044404450446044704480488
S11360D049044A044B044C044D044E044F04510437
S11360E052045304540455045604570458045904E0
S11360F05A045B045C045E045F0470217121722104
S113610073217421752176217721782179217A21CF
S11361107B217C217D217E217F2141FF42FF43FFA2
S113612044FF45FF46FF47FF48FF49FF4AFF4BFF37
S11361304CFF4DFF4EFF4FFF50FF51FF52FF53FFE7
S113614054FF55FF56FF57FF58FF59FF5AFF0000F1
S1136150C700FC00E900E200E400E000E500E7001D
S1136160EA00EB00E800EF00EE00EC00C400C5001C
S1136170C900E600C600F400F600F200FB00F900D6
S1136180FF00D600DC00A200A300A500A720920116
S1136190E100ED00F300FA00F100D100AA00BA001A
S11361A0BF001023AC00BD00BC00A100AB00BB00CD
S11361B091259225932502252425612562255625BE
S11361C055256325512557255D255C255B2510251F
S11361D0142534252C251C2500253C255E255F250A
S11361E05A25542569256625602550256C25672583
S11361F068256425652559255825522553256B2581
S11362006A2518250C25882584258C25902580252C
S1136210B103DF009303C003A303C303B500C403A6
S1136220A6039803A903B4031E22C603B5032922B7
S11362306122B1006522642220232123F700482231
S1136240B0001922B7001A227F20B200A025A000B6
S11362504100420043004400450046004700480016
S113626049004A004B004C004D004E004F005000C6
S11362705100520053005400550056005700580076
S113628059005A002100E0FFE1FFE5FFE2FFE3FFD0
S1136290C000C100C200C300C400C500C600C700DE
S11362A0C800C900CA00CB00CC00CD00CE00CF008E
S11362B0D000D100D200D300D400D500D600D8003D
S11362C0D900DA00DB00DC00DD00DE00780100012B
S11362D002010401060108010A010C010E0110016A
S11362E012011401160118011A011C011E012001DA
S11362F022012401260128012A012C012E0130014A
S113630032013401360139013B013D013F014101B4
S11363104301450147014A014C014E01500152011C
S11363205401560158015A015C015E016001620189
S11363306401660168016A016C016E0170017201F9
S11363407401760179017B017D019101910392032E
S113635093039403950396039703980399039A036D
S11363609B039C039D039E039F03A003A103A3031C
S1136370A403A503A603A703A803A903AA0310045F
S11363801104120413041404150416041704180445
S113639019041A041B041C041D041E041F042004F5
S11363A021042204230424042504260427042804A5
S11363B029042A042B042C042D042E042F04010484
S11363C0020403040404050406040704080409047D
S11363D00A040B040C040E040F04602161216221E1
S11363E063216421652166216721682169216A216D
S11363F06B216C216D216E216F2121FF22FF23FF70
S113640024FF25FF26FF27FF28FF29FF2AFF2BFF54
S11364102CFF2DFF2EFF2FFF30FF31FF32FF33FF04
S113642034FF35FF36FF37FF38FF39FF3AFF0000EE
S1096430FFFFFFFFFFFF68
S1056438010459
S90300F10B
